:020000040000FA
:100000008316FF2390009F01FC30850010308B0089
:100010008113951615158312073099000230A00040
:1000200085009F0105082039831601138312A10161
:10003000851A21140230A000850005088B1063008A
:10004000211832280130850000000230850041204F
:100050004120412000000000000005080439031978
:1000600022281A2801308500000000000230850097
:10007000412041204120412005080439031932283C
:100080001A280800493452342034523465346D340F
:100090006F347434653420345234653470346534CC
:1000A00061347434653472342E3420345034653401
:1000B00074346534203447347234693466346634B9
:1000C0006934743468347334203432343034303426
:1000D000343420342D34523465346D346F347434F8
:1000E0006534453478342D3434342E3461347334EB
:0200F0006D346D
:02400E00843FED
:00000001FF
